:100000000C9451050C946E050C946E050C946E05C1
:100010000C946E050C946E050C946E050C946E0594
:100020000C946E050C946E050C946E050C946E0584
:100030000C946E050C946E050C946E050C946E0574
:100040000C946E050C946E050C946E050C946E0564
:100050000C946E050C946E050C946E050C946E0554
:100060000C94FD080C946E050714371450146C148E
:100070009914C914E3141D1570510386400D4FEBFC
:100080003ECCD18735BDF50B5ED0F8F2D5E26C31B0
:100090000CADFC21C378C106C24C55E64A34481168
:1000A0001EDAE71A84A096A7E37FAF639CFA235B6E
:1000B00079C89EBAB2C922124BB3A1B63249A2E1A5
:1000C00089391066C5078F54EA91CA3FF919F0D7EC
:1000D00046BC281B61E82F6AAE9DF64E0914774D89
:1000E000DB1F2E7B7CF143A300B8138C85B92975E7
:1000F00088FDD2561C509741E53B60B5C064EE9830
:10010000D62D25A4AACD7DA883C6ABBE4499263C96
:10011000CE9FBFD3CB767A7E82018A9A801D0EB0A5
:100120005CD43862F430E08E53B70257ACA6520A62
:100130006D9265172433457274B1B4F75DED2CFFF1
:1001400047375A90BBDF2A165995D9C4276773C71A
:1001500068FEA5DD6B5F93D8EC053A8D6EFB3DA97B
:100160006936F394DEEF156F8B9B080FDC81182046
:1001700004E471CFE92B425801A0A962D63F85A7BC
:10018000B6D4FA15661709BD5D1434265972915418
:10019000064FF8B05B7493998CF245CDEA4EAD10E2
:1001A0004AE5CAEEDFC66F9F888E02CC08A8779416
:1001B0006D21B128E4397996607181162EE678B9FF
:1001C000C4469A42AEB77C43B3221A86C2323D2D52
:1001D0009CD229E9639BD131385E1E3641BB03189E
:1001E0002B3EBF6861FC52C0DEE00A58135A00BEC5
:1001F0001C900E5312FDE26EBACE2427447F87A3D3
:10020000A1D55040E3F983F7C7A235C8DB19AB2F5E
:100210001125ED339E55E148AF7384DA2AAA51EBDC
:100220009D95B2CBE77080FE4C6504EFC5F1C33AF3
:10023000B4F55F2389DD30A58BD3F6DC4D64D7F0B0
:100240008FEC56375CA40D07768A2C0BB5D8C11FEE
:10025000E83BF44B1B476C49677B92CF757E20D9F6
:100260007D3C977AD0056B0F1DFB8298578DF36A02
:10027000BCACC9A6FFB8690C4C4D72075A49338D06
:10028000A2AB463D630DA097FFF0F5FAC0E9DB6233
:10029000E4E17443DC86182937F406E2ED6F9048F8
:1002A0001E2D1DEA739454DF25F64727D91177C90F
:1002B000841C5B5C5181A6223E2496C88AEC827C19
:1002C00009B8454A57BB2F50758E61708C6CAFD002
:1002D000FDB41BAEDEFE3BB536BD55010E9C41564E
:1002E0005FB3260383BA134BCAC50AF860A5B9C722
:1002F000C39832FB12F9A792AA68F3787E052021F1
:1003000002E8BFF2B0598FD2CB876515F11AB2302F
:10031000ADEE58A38B661F2CD75D1985A8E6D36B6D
:10032000A10C91936A5E0B79E3DD004F3C896E71FD
:1003300069A9AC40E59928C6314E7ACD089E7DEF7B
:1003400017FC88D8A46D4495D1B7D49BBE2A3464D9
:100350002BCF2EEB38CE23E03A3FF77B9F1053BCD8
:10036000526716E7807604C4B6C1C27F9ADAD539DF
:1003700042149DB10F35D6CCB9DA380CA29C091FB6
:1003800006B1B6FD1A692330C4DE01D1F45829370D
:100390001C7DD5BFFFBDC8C9CF65BE7B7897986768
:1003A00008B32657F7FA40AD8E75A67CDB918B51CA
:1003B00099D4177A908DCE63CB4EA0AB183A5B5090
:1003C0007F2174C1BBB8B7BA0B359531599A4D042A
:1003D000071E5A7613F37183D08603A83942AA28E0
:1003E000E6E4D85DD3D06E6F96FB5EBC56C25F85E7
:1003F0009BE7AFD23B846AA753C54449A5F936723F
:100400003D2CD91BA1F54F939D68474116CA2A4C34
:10041000A387D6E5192E77156D70C0DFB20046EDC3
:10042000C66C4360922DA922458F3455AEA40A664E
:1004300032E0DC02ACE8208C89624AFEEEC3E33C89
:10044000F17905E9F62733CCF29E11817E80108A7E
:10045000829F480DD7B4FC2FB5C7DD88146B2B5491
:10046000EA1D945CB0EF1224CDEBE1E264733F0E21
:100470005261253EF80F4BECC00030F602493D10AA
:100480006E20C9A62FFE2C2B752E4526AB48A980C1
:10049000FC04CCD3B5BAA338317D01D9A77B96B67D
:1004A00063694EF7DEE078CA50AA41916588E4217D
:1004B00085DA3A27BE1C3E425E17527F1F89246FA1
:1004C0008F5C67740E12878DE934ED73C4F8615B3D
:1004D00005DF594C97798318A45595EBBD53F5F179
:1004E0005766469FB2810951862216DD23937629ED
:1004F000C2D71DD4BF363FEA4B1132B9625460D621
:100500006D439A0D929CB0EF586C9D772D70FAF365
:10051000B30BE2407EF48AE58C3C5671D164E182F3
:100520000ACB131590EC0399AF145D0F334A94A5D1
:10053000A8351BE36AC628FF4DE72584AC08AEC585
:10054000A22AB8370C7AA0C3CEAD061A9E8BFBD573
:10055000D0C11ED0B49BB144F247C768CF72BB4F25
:100560005AF9DC6BDBD2E87CC8EE98A1E6D83907F3
:100570005FFD8E19B73BBCCD7CE38173B211BF6FB9
:100580002098FE7596EF6CDA50E109725445BA3442
:10059000805BED3E532C87A457F3333F3CB767B4E1
:1005A000A325604F076B1B47150FE40AEAD1327889
:1005B00036498D4BD2BCA5DC1D0D4DCD9A825FFC1A
:1005C0009465BEE2F4C91E44CB9E0C64712663B3ED
:1005D00014E840708A0E19426DAC88105CDF41A9A6
:1005E000ADE5FB74CCD5068E5986CE1F3D76E08FE7
:1005F000B977277BA6D829D3ECB813F7FAC3516A89
:10060000DE4A5AEBC28B234892CF62A899F8D02ECB
:10061000856143C8BDF00593CA4EF17D30FDC469C4
:10062000662F08B152F921E67A2BDD3984FFC0919B
:10063000D637D47F2D9B5DA13B6EB5C54604F590A2
:10064000EE7E831C0356B6AA0017013555790B12AE
:10065000BB1A31E7022816C1F6A2DB189C8968385C
:1006600097ABC72AD73AF2C6244CB058A0225E9D59
:10067000D9A7E9AEAF8C959F28B720D7B030C30972
:1006800019C067D6003C7EE7E9F4085AF8B82E0591
:10069000A6259E5CD8150DE1F611546BCD2146665A
:1006A0005E84AD06382944C5A2CEF1AAC140718648
:1006B000B5EFFC36A8CB0A48274564A3AF8CB2C679
:1006C0009F0789DC17D34979FBFE1DD0B9884352B7
:1006D000BC01782B7D94C70EDEA5D59BCCF7617A43
:1006E000C274813903AB96A037BD2D72753FC9D452
:1006F0008E6FF98DED62DB1CDF04AC1B6C144B6359
:10070000D0BFB482EC7B1A5992D21060B63D5FE63E
:10071000806E70C4F235D97CEEE541A45B50DDBB40
:100720004CF31F9D5D57555197E358424D9C73BA4A
:10073000C877316926AEEA8ADA22B38756FA930B74
:10074000341633E8E453BEA9B13A3EF5906ACF3B84
:1007500012FD8F9AA7479199EB0F24FF2318854E1E
:100760007F0CE0A1D2D12C2A4A024F1E95688B98AB
:10077000836D76CA6532132FC3829AA4BA8160371B
:100780003435FC80A8516567ED305F10D34A272FC0
:1007900013B92AD2CCE1EFAEEBBEF4BDCF43B3C563
:1007A0008884B7DD3940CE486D9B72617EE7A14EEB
:1007B000532E773BE2C936221B6E73B103B24C87CE
:1007C000A9D44D0FD8156CAA18F649575DFB7A14B9
:1007D0009463A011B09EDE0546C8EE47DBDC248999
:1007E0009C919729E97BC1071EB8FDFEACC66298B3
:1007F0004FF179E0E86B7856B68D045086CA6F20C9
:10080000E6EAE576171C747FBC0D2C85F76696E446
:100810008B753F4BD938AF7CDA0B832D3132A2F583
:100820001D594145BF3C1FF8F98AD0162569129918
:100830009D2195AB01A6D7B5C07DFF580E3A92D148
:1008400055E3089FD63E528EFAA3C702CDDF8F64D0
:10085000198CF3A70C5E0A6A09F0935B42C2062367
:10086000EC71ADB4CBBB7028D51A5C33685A004428
:1008700090A5C4263D2BF25496ADDA1FED33E181ED
:1008800069080D0ADB35779A64D1FC78AA1BD0671A
:10089000A0DDFA6C63710584176A894F667FC650C4
:1008A00055926FBDE7D240728DBBEC06428AE48858
:1008B0009D7E7A822713411AAFC8A476B4C2FE6D1A
:1008C0001CD96130B37CEAF7290FF23B51C1DE5FDE
:1008D000E52A2F990B5DA32B4AAB95A5D35856EE6D
:1008E000283100CC1546CAE686383C65F5E39FD62C
:1008F0005B094983702D53A97DE2C4AC8E5EB82597
:10090000F4B957F3F16847B2A25920CE34795C901C
:100910000E1EBED52223B1C91862162E913E078F36
:10092000D83F933DD49BDF8521FB117497C7D7DC5B
:100930004C194598E943024BBCC3049C6BF07552BB
:10094000A726F6C5BACFB0B7AE5AA1BF038B8012A7
:100950006E0CEBF9C04424EF10F8A88CE87BFF9EE6
:100960002CCD603687B594A654733A144E011DB64B
:10097000FD37484D39CBE032000000000000000098
:100980000000000000000000000000000000000067
:100990000000000000000000000000000000000057
:1009A0000000000000000000000000000000000047
:1009B0000000000000000000000000000000000037
:1009C0000000000000000000000000000000000027
:1009D0000000000000000000000000000000000017
:1009E0000000000000000000000000000000000007
:1009F00000000000000000000000000000000000F7
:100A000000000000000000000000000000000000E6
:100A100000000000000000000000000000000000D6
:100A200000000000000000000000000000000000C6
:100A300000000000000000000000000000000000B6
:100A400000000000000000000000000000000000A6
:100A50000000000000000000000000000000000096
:100A60000000000000000000000000000000000086
:100A70000000000000000000A877A6E0F7435A3508
:100A800085E272978FB71A6287380D67C7BE4F3EEF
:100A90002076378F68B7A9263F2B10E3307E900E63
:100AA000850A11241FBECFEFD4E0DEBFCDBF11E019
:100AB000A0E0B1E0EAE0F5E302C005900D92A83EA7
:100AC000B107D9F724E0A8EEB1E001C01D92AF391B
:100AD000B207E1F70E948C180C94831A0C94000062
:100AE00081E08093EA010895E82FF0E0E250FE4FA4
:100AF00080810895882311F085EC01C085E88093FA
:100B0000BC000895482F50E028E030E0261B310952
:100B1000CA01022E01C0880F0A94EAF702C0559557
:100B200047956A95E2F7842B08952F923F924F9252
:100B30005F926F927F928F929F92AF92BF92CF926D
:100B4000DF92EF92FF920F931F93CF93DF93CDB776
:100B5000DEB7E2970FB6F894DEBF0FBECDBF1DA67D
:100B60001CA6A12CB12C78E0E72EF12CDE015196C9
:100B700080E090E02CA53DA52858354FF901E80FFD
:100B8000F91FE491ED93019686309105B9F7DE01E6
:100B9000119680E090E0FC01EC5EFC4FE081F0E01B
:100BA000E858FF4FE491ED9301968A30910599F74B
:100BB000AB817E818989872790E04A2F47702A85FB
:100BC00028ABFD819701241B31093AAB29AB9C016D
:100BD00009A802C0220F331F0A94E2F702C09595BC
:100BE00087954A95E2F7822B38A9831B8F278B873D
:100BF000B9814A814EA78A89842790E04B2F47709C
:100C0000E8859701241B31093AAB29AB9C0109A85F
:100C100002C0220F331F0A94E2F702C09595879510
:100C20004A95E2F7822B871B8E278C873F813FA74F
:100C30002B89232730E069856770C701861B9109DE
:100C4000A901082E01C0440F0A94EAF7062E02C03B
:100C5000359527950A94E2F7242B2A1B2B272D87FD
:100C60002C892F2730E04E2F47704BA79C81A7017E
:100C7000BBA54B1B51095AAB49ABA90109A802C03E
:100C8000440F551F0A94E2F702C035952795BA958F
:100C9000E2F7242B291B2A272E872D895EA52527DD
:100CA00030E0AFA5A770A7014A1B51095AAB49AB69
:100CB000A90109A802C0440F551F0A94E2F75AABD4
:100CC00049AB02C035952795AA95E2F7242B291B3D
:100CD0002F272F872E892E2730E0F90102C0EE0F33
:100CE000FF1F8A95E2F7CF0102C0359527956A95D7
:100CF000E2F7822B871BF8A98F27888B46E050E00C
:100D00006EE073E0CE010B960E94341A95012F5FBE
:100D10003F4F892B79F059012CA53DA52A5F3F4F04
:100D20003DA72CA737E0A316B10409F01FCF1092FE
:100D30001E0380C1822F90911203122F00E0090F31
:100D4000111D08581F4FF8010491F2E0AF0EB11CBD
:100D500090911703FA2DEE27E90FF11DE858FF4F88
:100D6000E491E027E093060390911003782E612C24
:100D7000690E711C930128583F4FF90164909091BE
:100D80001903FA2DEE27E90FF11DE858FF4FE49102
:100D9000E625E093070390911303582E412C490E4A
:100DA000511C920128583F4FF901449090911B0328
:100DB000FA2DEE27E90FF11DE858FF4FE491E425E5
:100DC000E093080390910E03D82EC12CC90ED11CBC
:100DD000960128583F4FF901949120911603FA2D5E
:100DE000EE27E20FF11DE858FF4FE491E927E09369
:100DF000090390910F03982E812C890E911C940168
:100E000028583F4FF901949120911803FA2DEE27AD
:100E1000E20FF11DE858FF4FE491E927E0930A0340
:100E200090911103888F1F8A2F89388D290F311DCA
:100E300028583F4FF901949120911D03FA2DEE2778
:100E4000E20FF11DE858FF4FE491E927E0930B030F
:100E5000909114038A8F198E298D3A8D290F311D97
:100E600028583F4FF901949120911A03FA2DEE274B
:100E7000E20FF11DE858FF4FE491E927E0930C03DE
:100E8000909115038C8F1B8E2B8D3C8D290F311D5E
:100E900028583F4FF901949120911C03FA2DEE2719
:100EA000E20FF11DE858FF4FE491E927E0930D03AD
:100EB00090910E038E8F1D8E2D8D3E8D290F311D2D
:100EC00028583F4FF901949120911503FA2DEE27F0
:100ED000E20FF11DE858FF4FE491E927E093FE028D
:100EE0009091130388A31F8E2F8D38A1290F311DD8
:100EF00028583F4FF901949120911803FA2DEE27BD
:100F0000E20FF11DE858FF4FE491E927E093FF025B
:100F1000909111038AA319A229A13AA1290F311D89
:100F200028583F4FF901949120911403FA2DEE2790
:100F3000E20FF11DE858FF4FE491E927E093000329
:100F4000909110038CA31BA22BA13CA1290F311D52
:100F500028583F4FF901949120911D03FA2DEE2757
:100F6000E20FF11DE858FF4FE491E927E0930103F8
:100F7000909112038EA31DA22DA13EA1290F311D18
:100F800028583F4FF901949120911B03FA2DEE2729
:100F9000E20FF11DE858FF4FE491E927E0930203C7
:100FA00090910F0388A71FA22FA138A5290F311DEB
:100FB00028583F4FF901949120911C03FA2DEE27F8
:100FC000E20FF11DE858FF4FE491E927E093030396
:100FD000909117038AA719A629A53AA5290F311DB3
:100FE00028583F4FF901949120911903FA2DEE27CB
:100FF000E20FF11DE858FF4FE491E927E093040365
:1010000090911603382E212C290E311C910128585D
:101010003F4FF901249080911A03FA2DEE27E80F33
:10102000F11DE858FF4FE491E225E093050381E0CC
:1010300080931E03E2960FB6F894DEBF0FBECDBFBD
:10104000DF91CF911F910F91FF90EF90DF90CF90A4
:10105000BF90AF909F908F907F906F905F904F90D8
:101060003F902F900895863028F4E0911F03F0916F
:1010700020030994089590EC980F963098F480E43A
:1010800090E029E430E0F901E81BF90BDC01A25003
:10109000BE4F4C91EC5EFC4F408301968634910527
:1010A00091F708959AEB980F9630C8F48091440216
:1010B0008093170380914502809316038091460226
:1010C0008093150380914702809314038091480216
:1010D000809313038091490280931203089594EB47
:1010E000980F9430C0F490914A029093110390911C
:1010F0004B029093100390914C0290930F039091A8
:101100004D0290930E0370E0680F711D60357105FC
:1011100011F40C9495050895462F50E0BC018EEF14
:1011200091E00C94411AEF92FF920F931F93CF938B
:10113000DF9300D0CDB7DEB77C01CB011093200345
:1011400000931F03642F29833A830E948C08109216
:10115000EE0286E0F701ACEEB1E001900D928A95C7
:10116000E1F786E0ECEEF1E0A8EFB2E001900D923D
:101170008A95E1F72981E22F3A81F32F80E290E00E
:101180002191DC01A250BE4F2C9301968034910531
:10119000B9F7459844981092FD011092FC0184EA39
:1011A0008093BA0081E48093BC000F900F90DF9190
:1011B000CF911F910F91FF90EF9008958091EB01D7
:1011C00008958091EB01811108C08091BC0084607A
:1011D0008093BC0081E08093EB0108958091F80139
:1011E000089526E0FC01A2EFB1E001900D922A954E
:1011F000E1F781E08093F90108951F920F920FB6F5
:101200000F9211242F933F934F935F936F937F938C
:101210008F939F93AF93BF93EF93FF938091B90008
:10122000887F803951F188F4803721F128F48036A5
:1012300009F18836F9F0D4C08038F9F0883809F41B
:10124000CFC0883709F0CCC015C0803B09F48DC0F1
:1012500038F4803A09F47DC0883A09F0C1C085C0ED
:10126000803C09F4BBC0883C09F4B8C0883B09F451
:1012700084C0B6C01092FB01B1C08091FB018823ED
:1012800009F45AC02091BB008091FC019091FD01AE
:10129000803F910589F4253511F02A3A69F41092BE
:1012A0001E0386E0ECEEF1E0A8EFB2E001900D92B3
:1012B0008A95E1F71092F8018091FC019091FD016F
:1012C000892B91F4243681F48091F901882361F00F
:1012D00086E0E2EFF1E0A8EFB2E001900D928A958E
:1012E000E1F781E08093F80180911E038823E1F00B
:1012F000A091FC01B091FD01E091FC01F091FD0194
:10130000E770FF27E250FD4F8081E091FC01F091F2
:10131000FD01E770FF27EA5FFC4F90818227890F6C
:10132000A250BE4F8C934CC0E091FC01F091FD01A6
:10133000E250FE4F208344C08091BB0090E0909328
:10134000FD018093FC0181E08093FB011092FA0182
:1013500045C06091FA018091FC019091FD0190914E
:10136000FA01891B0E943B0839C08091FC019091D1
:10137000FD010E9433081092FA0180911E03E09152
:10138000FC01F091FD01E250FE4F8823B1F0808115
:10139000E091FC01F091FD01E770FF27EA5FFC4F4F
:1013A0002081E091FC01F091FD01E770FF27E25000
:1013B000FD4F9081821B892701C080818093BB00F3
:1013C0008091FC019091FD0101969093FD01809325
:1013D000FC018091FA018F5F8093FA0185EC01C0D6
:1013E00085E88093BC00FF91EF91BF91AF919F91F1
:1013F0008F917F916F915F914F913F912F910F90BE
:101400000FBE0F901F901895FC01009701F12091DD
:10141000240330912503832F8F708F3021F481E0D6
:101420008093210302C0109221038091210388231D
:1014300029F083E080832183228309C082E08083B6
:10144000822F90E0932B9283818323833483809136
:1014500024039091250390932303809322030895FE
:1014600042E050E062E273E084E293E00E94341ACA
:101470000895419A30E33A95F1F7419888E090E079
:1014800020E038E13A95F1F74098220F329B216035
:1014900038E13A95F1F7409A0197009791F7209338
:1014A000240388E090E038E13A95F1F74098220F64
:1014B000329B216038E13A95F1F7409A0197009705
:1014C00091F72093250380E00895CF93CFB7F89448
:1014D000399A389A3A98429A409A41980E94390A21
:1014E000CFBF80E0CF9108958EE391E008958823E7
:1014F000C9F091E0E82FFF27E7FDF095292F30E0B4
:10150000241735076CF4DB01A20FB31F2C9130E0D8
:10151000E217F3071CF48FEF890F08959F5FEECF5A
:101520008FE1089580E0089540E250E0623041F09C
:10153000633019F06AE871E005C06AE671E002C044
:101540006AE471E00C94770A009741F023E1E9E343
:10155000F3E0DC0101900D922A95E1F783E1E9E3E4
:10156000F3E0A6E2B3E001900D928A95E1F70895C9
:101570002091B601253069F0222359F0892B21F002
:10158000233039F082E003C0213019F084E08093E9
:10159000B60108951F93CF93DF931F92CDB7DEB7A7
:1015A00085E08093B6011FE02FE389E191E02150AF
:1015B00080409040E1F700C00000198261E070E0D7
:1015C000CE0101960E94270C489721F0115061F737
:1015D00080E001C081E00F90DF91CF911F910895CD
:1015E00043E150E066E273E089E393E00E94341A3D
:1015F00008951F93CF93DF93CDB7DEB7A6970FB6AD
:10160000F894DEBF0FBECDBF198261E070E0CE015D
:1016100001960E94270C883119F01092B60100C182
:101620008091B203882331F08091B601853011F4A6
:101630001092B6018091B203811103C085E08093BE
:10164000B6018091B6018230E1F0843099F18111C8
:1016500049C083E0898380E88A8381E08B8342E20A
:1016600050E060E870E0CE0104960E944A1A63E2FE
:1016700070E0CE0101960E94270C882399F184E046
:101680002FC013E0198380EC8A838BE18B8340E2C7
:1016900050E061E070E0CE0104960E944A1A63E2D5
:1016A00070E0CE0101960E94270C8823D9F0109398
:1016B000B60118C083E0898380EC8A838BE18B8339
:1016C000FE01349680E2DF011D928A95E9F763E21C
:1016D00070E0CE0101960E94270C882319F081E06A
:1016E0008093B60181E0898361E070E0CE010196CC
:1016F0000E94270C803209F093C084E08093390364
:1017000020E030E080E090E041E050E0FC01E55670
:10171000FC4F6081662349F0BA01082E02C0660FB3
:10172000771F0A94E2F7262B372B0196803191051B
:1017300069F730933D0320933C0319821A8260E0DD
:1017400080E090E020E830E0FC01E555FC4F40816E
:10175000442341F0A901082E02C0559547950A94EB
:10176000E2F701C040E0642B01968830910561F7F3
:1017700069837A8180E090E020E830E0FC01ED545C
:10178000FC4F4081442341F0A901082E02C0559529
:1017900047950A94E2F701C040E0472B0196883054
:1017A000910511F0742FEACF4A8360933A03409376
:1017B0003B03603819F481E880933A03403819F408
:1017C00081E880933B0310923E0310923F031092F6
:1017D00040031092410380E090E020E830E0FC01FB
:1017E000E556FC4F40814423A9F0FC0143E0F59508
:1017F000E7954A95E1F7E75CFC4FAC014770552748
:10180000B90102C0759567954A95E2F7AB0155811C
:10181000542B558301968032910509F780E001C071
:101820008FEFA6960FB6F894DEBF0FBECDBFDF9147
:10183000CF911F9108950E94F90A80E008958AEAE5
:1018400091E008953B984398249A2C9808950F931B
:101850001F93CF93DF93662309F44FC07727A0E04F
:10186000B0E040E050E09D0146175707ACF41896F1
:1018700010E8FC01E40FF51F00810123E901C556C2
:10188000DC4F08832F5F3F4F16952A173B07A1F7C0
:101890004F5F5F4FD901E7CFEBE9F3E0CF93DF93E1
:1018A000EF93FF930191002311F049F416C000005B
:1018B0003B9A19E00FD03B981197A1F70EC03B9AC5
:1018C00011E008D03B9815E005D00000000011970A
:1018D00049F703C01A95F1F708950000FF91EF91C1
:1018E0003B9ADF91CF9100000000000000003B9880
:1018F0000FEF0A9511F0339BFCCFEBE9F3E0EF9388
:10190000FF93442700270395A1F03399FCCF08C02B
:1019100004E6039572F03399FCCF439551F001939F
:1019200004E6039532F0339BFCCF439511F001930D
:10193000EFCFFF91EF91842F90E00097B9F040FF37
:1019400015C0DF019D017081618151E0761708F0BB
:1019500050E05D9332965A2F521B5417A0F324E1A6
:101960002A95F1F701979595879502C080E090E060
:10197000DF91CF911F910F910895CF93DF931F9225
:10198000CDB7DEB7198261E070E0CE0101960E940A
:10199000270C0097F1F04897F9F480919F0381118B
:1019A00088E09091A003911184609091A10391111E
:1019B00082609091A203911181608A3038F488305E
:1019C00070F4853049F481E090E00BC08B3039F041
:1019D00003C080E090E005C083E090E002C082E0B8
:1019E00090E00F90DF91CF910895009741F023E1AF
:1019F000E4E6F3E0DC0101900D922A95E1F7089509
:101A000043E150E061E573E084E693E00E94341A1C
:101A1000089585E08093640320E030E080E090E06A
:101A200041E050E0FC01E556FC4F6081662349F03F
:101A3000BA01082E02C0660F771F0A94E2F7262B20
:101A4000372B01968031910569F730936C03209311
:101A50006B0360E080E090E020E830E0FC01E555B9
:101A6000FC4F4081442341F0A901082E02C0559546
:101A700047950A94E2F701C040E0642B0196883054
:101A8000910561F7B0E080E090E020E830E0FC01F3
:101A9000ED54FC4F4081442341F0A901082E02C0BF
:101AA000559547950A94E2F701C040E0B42B0196A2
:101AB0008830910561F770E080E090E020E830E048
:101AC000FC01E554FC4F4081442341F0A901082E5C
:101AD00002C0559547950A94E2F701C040E0742B87
:101AE00001968830910561F770936703A0E080E06C
:101AF00090E020E830E0FC01ED53FC4F40814423AE
:101B000041F0A901082E02C0559547950A94E2F7C5
:101B100001C040E0A42B01968830910561F78091C7
:101B200050038823A9F080914F03681B60936503DD
:101B300080914E03B81BB093660380914D03781BD0
:101B40007093670380914C03A81BA093680313C094
:101B500060934F03B0934E0370934D03A0934C03D7
:101B60001092650310926603109267031092680347
:101B700081E08093500380E090E060E020E830E076
:101B8000FC01E553FC4F4081442341F0A901082E9C
:101B900002C0559547950A94E2F701C040E0642BD6
:101BA00001968830910561F76093690380E090E0C9
:101BB00060E020E830E0FC01ED52FC4F408144231E
:101BC00041F0A901082E02C0559547950A94E2F705
:101BD00001C040E0642B01968830910561F7609365
:101BE0006A0388E0EDE6F3E0DF011D928A95E9F7EC
:101BF00080E090E020E830E0FC01E556FC4F4081B9
:101C00004423A9F0FC0143E0F595E7954A95E1F7F7
:101C1000EC59FC4FAC0147705527B90102C07595CE
:101C200067954A95E2F7AB015185542B5187019690
:101C30008034910509F70895CF93DF93CDB7DEB7D0
:101C400028970FB6F894DEBF0FBECDBF80E489831E
:101C500083E08A831B8263E070E0CE0101960E94DC
:101C6000270C803421F40E94090D80E001C081E03E
:101C700028960FB6F894DEBF0FBECDBFDF91CF918F
:101C80000895109250030E941C0E91E0811190E083
:101C9000892F08950E941C0E80E0089587EB91E043
:101CA00008958EE0E3ECF1E0A8E7B3E001900D9237
:101CB0008A95E1F74EE050E060E070E088E793E05D
:101CC0000C94611A4EE050E060E070E088E793E029
:101CD0000E94511A49E050E06EED71E088E793E010
:101CE0000E94341A892BD1F08EE0E8E7F3E0DF019F
:101CF0001D928A95E9F789E0EEEDF1E0A8E7B3E0FF
:101D000001900D928A95E1F74EE050E060E070E0BE
:101D100088E793E00E94611A0C94510E8EE0E8E788
:101D2000F3E0A3ECB1E001900D928A95E1F70895FC
:101D300020917703211104C0FC0160830C94510EA3
:101D40000895FF920F931F93CF93DF93EC018B01C4
:101D500081E1FB0111928A95E9F741305105A9F41F
:101D60008091CC01883059F06091CD0170E089817B
:101D70000E94AF16F82E6091CD0170E011C0F9807D
:101D8000F0E2FF0E8A81805E25C04230510561F489
:101D900062E070E089810E94AF16F82E62E070E088
:101DA0008A810E94AF1616C08981992787FD909578
:101DB00080589F4F9595879595958795F82E2A8100
:101DC000332727FD309520583F4F3595279535957A
:101DD0002795822F2B81332727FD309520583F4FA1
:101DE00093E0359527959A95E1F74C81552747FD66
:101DF000509540585F4F63E0559547956A95E1F7D8
:101E00009D819595959595955E81B901E3E0660F65
:101E1000771FEA95E1F7607C6F29F8016083B901CB
:101E2000A5E0660F771FAA95E1F7607C682B6183B8
:101E30003695322F222737952795692F6871F4E060
:101E40006F9FB0011124262B242BF8012283F0E28E
:101E50009F9FC0011124569556955695582BF80111
:101E600053838885809584838F818095858382E5DF
:101E7000868389859A8590878783D8011996FE0184
:101E80003B9688E001900D928A95E1F7DF91CF9122
:101E90001F910F91FF900895CF93DF93DC01FB0119
:101EA00081E1EB0119928A95E9F712969C911297BC
:101EB000905813962C911397205814968C91149740
:101EC000805815965C91159716964C911697119619
:101ED0003C911197305830832183928383831482FD
:101EE0005583468318968C9118978095878317960B
:101EF0008C9180958087DF91CF910895CF93DF9368
:101F0000DC01FB0181E1EB0119928A95E9F7129658
:101F10009C911297905813962C91139720581496D1
:101F20008C911497805815965C91159716964C9144
:101F3000169711963C9111973058308321839283E4
:101F400083835483458318968C9118978095868354
:101F500017968C9180958783DF91CF9108952130DA
:101F6000310539F02230310511F00C94A10E0C949A
:101F70007E0F0895EF92FF920F931F93CF93DF93FD
:101F80007C01EB0183E1DB011D928A95E9F7F70102
:101F90008081843009F473C330F4823069F0833077
:101FA00009F4EEC0D5C6863009F442C608F43EC135
:101FB000873009F405C6CCC683E5898786E48A871D
:101FC000838194819C878B879091CF018181992314
:101FD00079F086FF05C08F819885806498878F830C
:101FE000F701818187FF2BC08F819885806125C093
:101FF00087FF05C08F819885806498878F83D7017C
:1020000011968C9186FF05C08F8198858062988794
:102010008F83F7018181928197FF05C08F81988519
:10202000806198878F83D70111968D919C9112972B
:1020300096FF05C08F819885886098878F839091DF
:10204000D001F70181819923C9F083FF02C084E6A2
:102050008A83D70111968C9182FF02C08CE98A8312
:10206000F701818181FF02C08CE98983D701119634
:102070008C9180FF26C084E6898323C083FF05C03E
:102080008F819885816098878F83F701818182FF96
:1020900005C08F819885906498878F83D7011196AA
:1020A0008C9181FF05C08F819885826098878F838E
:1020B000F701818180FF05C08F819885906898879E
:1020C0008F83D70111968C9185FF05C08F819885EC
:1020D000906198878F83F701818184FF05C08F818C
:1020E0009885946098878F83D70111968D919C91E4
:1020F000129795FF05C08F819885906298878F838E
:10210000F7018181928194FF05C08F81988592604B
:1021100098878F83D70111968D919C911297887320
:1021200090738833904331F41092CF011092D00114
:102130000E94510EF70181819281847390738433E0
:10214000904339F481E08093CF011092D0010E9436
:10215000510ED70111968D919C91129782739073B5
:102160008233904339F481E08093D0011092CF0103
:102170000E94510EF70181819281807199270CC5CF
:1021800086E4898783E48A8782818B87818187FFC0
:1021900005C08F819885806198878F83F701818141
:1021A00086FF05C08F819885806498878F83D701CB
:1021B00011968C9185FF05C08F81988590619887D5
:1021C0008F83F701818184FF05C08F81988594609A
:1021D00098878F83D70111968C9183FF05C08F81DB
:1021E0009885816098878F83F701818182FF05C080
:1021F0008F819885906498878F83D70111968C91F1
:1022000081FF05C08F819885826098878F83F70151
:10221000818180FF05C08F819885906898878F8322
:10222000D70111968C91807190E07FC587E48987F2
:1022300083E48A8788E0F7013996DB011B960190D9
:102240000D928A95E1F7F7018781442329F083FFF6
:1022500003C091E0909377039091CE01923009F4FE
:102260007FC028F4992361F09130B9F183C1943093
:1022700009F4F9C008F4B4C0953009F437C17AC143
:1022800087FF05C08F819885806198878F83D701EC
:1022900017968C9186FF05C08F81988580649887FA
:1022A0008F83F701878185FF05C08F8198858860BE
:1022B00098878F83D70117968C9184FF05C08F81F3
:1022C0009885806298878F83F7018781908593FF37
:1022D00032C08F81988584682CC086FF05C08F81AD
:1022E0009885806298878F83D70117968C9187FF96
:1022F00005C08F819885806498878F83F7018781D7
:1023000084FF05C08F819885886098878F83D70167
:1023100017968C9185FF05C08F819885806198877D
:102320008F83F7018781908593FF05C08F81988502
:10233000906198878F83D70117968D919C911897FC
:1023400091FF05C08F819885906298878F83F701F0
:102350008781908592FF0EC18F819885926008C118
:1023600087FF05C08F819885806198878F83D7010B
:1023700017968C9186FF05C08F8198858064988719
:102380008F83F701878185FF05C08F8198858860DD
:1023900098878F83D70117968C9184FF05C08F8112
:1023A0009885806298878F83F7018781908593FF56
:1023B00005C08F819885926098878F83D701179683
:1023C0008D919C91189791FF05C08F8198858068A9
:1023D00098878F83F7018781908592FFCBC082C059
:1023E00087FF05C08F819885846098878F83D70188
:1023F00017968C9186FF05C08F819885806198879C
:102400008F83F701878185FF05C08F819885806460
:1024100098878F83D70117968C9184FF05C08F8191
:102420009885886098878F83F7018781908593FFCF
:1024300005C08F819885806498878F83D701179610
:102440008D919C91189791FF05C08F819885806828
:1024500098878F83F7018781908592FF8BC08F814A
:102460009885806285C087FF05C08F8198858064CC
:1024700098878F83D70117968C9186FF05C08F812F
:102480009885806298878F83F701878185FF05C0D3
:102490008F819885806198878F83D70117968C915B
:1024A00084FF05C08F819885886098878F83F701A6
:1024B0008781908591FF05C08F819885906298876C
:1024C0008F83D70117968D919C91189792FF05C025
:1024D0008F819885926098878F83F7018781908597
:1024E00093FF48C08F819885846042C087FF05C0F4
:1024F0008F819885806198878F83D70117968C91FB
:1025000086FF05C08F819885886098878F83F70143
:10251000878185FF05C08F819885926098878F831A
:10252000D70117968C9184FF05C08F8198858064B0
:1025300098878F83F7018781908591FF05C08F81F0
:102540009885806898878F83D70117968D919C9185
:10255000189792FF05C08F819885846098878F8334
:10256000F7018781908593FF05C08F8198859061E1
:1025700098878F83D70117968C9183FF05C08F8131
:102580009885946098878F83F7018781908594FF61
:1025900005C08F819885816098878F83D7011796B2
:1025A0008D919C91189795FF05C08F8198859064B7
:1025B00098878F83F7018781908597FF05C08F816A
:1025C0009885826098878F83D70117968D919C910B
:1025D000189796FF05C08F819885906898878F839C
:1025E000F7018181898382818A8383818B838481BE
:1025F0008C8385818D8386818E83878190859C01E4
:10260000207F3071203F304111F460E02CC09C01EC
:10261000207F3072203F304211F461E024C09C01E1
:10262000207F3078203F304811F462E01CC09C01CC
:10263000207F3074203F304411F463E014C0807F69
:102640009870803F984099F4D70113968C91803C04
:102650002CF464E08EEC91E00E94980EF7018381E7
:1026600081342CF065E08EEC91E00E94980ED70149
:1026700017968D919C9118978870992756C386E379
:10268000898784E38A87F701058116812781308550
:102690000B871C872D873E8783819481442329F0F3
:1026A00083FF03C021E0209377039C0124713C70D9
:1026B00024313C4011F460E036C09C0124723C702F
:1026C00024323C4011F461E02EC09C0124743C7023
:1026D00024343C4011F462E026C09C0124783C7014
:1026E00024383C4011F463E01EC09C0124703C710E
:1026F00024303C4111F464E016C09C0124703C720B
:1027000024303C4211F465E00EC09C0124703C74FE
:1027100024303C4411F466E006C084709C78843018
:102720009C4829F467E08CEC91E00E94980E80911F
:102730007703811115C0F701838194819C01257075
:102740003C7025303C4011F483E006C086709C70DC
:1027500086309C4029F481E08093CD010E94510E87
:10276000D70113968C9180FF05C08F819885806179
:1027700098878F83F701838181FF05C08F819885BA
:10278000806498878F83D70113968C9183FF05C04F
:102790008F819885946098878F832091CC01283011
:1027A000B1F1F701838184FF05C08F819885816035
:1027B00098878F83D70113968C9185FF05C08F81F1
:1027C0009885906498878F83F701838186FF05C081
:1027D0008F819885826098878F83D70113968C911B
:1027E00087FF05C08F819885906898878F83422FD7
:1027F00050E04830510508F03FC1FA01EC5CFF4F52
:10280000D70113968D919C9114970C942E1AF70171
:10281000838182FF05C08F819885846898878F8324
:10282000D70113968D919C91149793FF05C08F81CA
:102830009885926098878F83F7018381948192FFB6
:1028400005C08F819885906298878F83D7011396F2
:102850008D919C9114978474907F8434904F09F0EB
:1028600009C18F819885886298878F8303C182FF11
:1028700005C08F819885906298878F83F701838147
:10288000948193FF05C08F819885926098878F838C
:10289000D70113968D919C91149792FFEDC0C9C0FA
:1028A00082FF05C08F819885906298878F83F7019A
:1028B0008381948193FF05C08F819885926098876A
:1028C0008F83D70113968D919C91149792FFD4C05A
:1028D0008F8198859064CBC092FF05C08F819885C9
:1028E000906498878F83F7018381948193FF05C05B
:1028F0008F819885846898878F83D70113968C91F0
:1029000082FF05C08F819885926298878F83F70137
:102910008381948196FF05C08F8198858062988716
:102920008F83D70113968D919C91149795FFA4C026
:102930002CC092FF05C08F819885846898878F830B
:10294000F7018381948193FF05C08F819885926000
:1029500098878F83D70113968C9182FF05C08F8152
:102960009885906298878F83F7018381948196FF81
:1029700005C08F819885806298878F83D7011396D1
:102980008D919C91149797FF77C08F81988588606F
:102990006EC092FF05C08F819885906298878F8363
:1029A000F7018381948193FF05C08F8198859260A0
:1029B00098878F83D70113968C9182FF5DC08F819A
:1029C0009885906254C092FF05C08F819885906869
:1029D00098878F83F7018381948193FF05C08F814E
:1029E0009885926098878F83D70113968C9182FF88
:1029F00005C08F819885906298878F83F7018381C6
:102A0000948195FF05C08F819885886098878F8312
:102A1000D70113968D919C91149796FF05C08F81D5
:102A20009885806298878F83F7018381948197FFCF
:102A300023C08F81988584681AC092FF05C08F815A
:102A40009885846898878F83D70113968D919C9180
:102A5000149793FF05C08F819885926098878F8324
:102A6000F701838182FF08C08F81988588629887EB
:102A70008F8302C0283039F1243009F460C1263038
:102A800009F45DC1D70113968D919C91149794FF21
:102A900002C084E68C83F7018381948195FF02C094
:102AA0008CE98C83D70113968D919C91149796FF96
:102AB00002C08CE98B83F7018381948197FF3FC12A
:102AC00084E68B833CC1D70113968D919C9114971A
:102AD0002091880394FF09C020FD0AC0309187032C
:102AE0003F5F30938703216001C02E7F20938803CE
:102AF0002091880395FF09C021FD0AC0309187030A
:102B0000315030938703226001C02D7F20938803CA
:102B10002091880396FF09C022FD0AC030918603E8
:102B20003F5F30938603246001C02B7F209388038E
:102B30002091880397FF09C023FD0AC030918603C6
:102B4000315030938603286001C0277F209388038B
:102B500084FF03C0809187038A83F701838185FF07
:102B600004C08091870381958A83D70113968C9145
:102B700086FF03C0809186038983F701838187FFE5
:102B800004C08091860381958983D70113968D9126
:102B90009C911497887099270E94F216882329F037
:102BA0008F819885986098878F838F81988595FF0E
:102BB00002C02FEF2D8391FFCBC08FEF8E83C8C053
:102BC000F701818180FF05C08F819885816098879A
:102BD0008F83D70111968C9181FF05C08F819885D5
:102BE000906498878F83F701818182FF05C08F8170
:102BF0009885826098878F83D70111968C9183FF87
:102C000005C08F819885906898878F83F7018181AF
:102C100084FF05C08F819885806498878F83D70152
:102C200011968C9185FF94C08F819885806184C0B6
:102C3000F701818180FF05C08F8198858160988729
:102C40008F83D70111968C9181FF05C08F81988564
:102C5000906498878F83F701818182FF05C08F81FF
:102C60009885826098878F83D70111968C9183FF16
:102C700005C08F819885906898878F83F70181813F
:102C800086FF05C08F819885806298878F83D701E2
:102C900011968C9184FF05C08F81988580649887F8
:102CA0008F83F701818185FF05C08F8198858061C1
:102CB00098878F83D70111968C9187FF05C08F81EC
:102CC0009885906298878F83F7018181928190FF28
:102CD00005C08F819885886098878F83D70111966A
:102CE0008D919C91129791FF05C08F81988592607C
:102CF00098878F83F7018181928192FF05C08F8130
:102D00009885946098878F83D70111968D919C91B7
:102D1000129793FF05C08F819885846098878F8371
:102D2000F70181819281882794700E94F21688238E
:102D300079F08F819885986098878F8309C0D70133
:102D400011968C911197898312968C918A831DCF4D
:102D5000DF91CF911F910F91FF90EF90089587FD24
:102D600005C00E94940A90E2980F05C081950E94C8
:102D7000940A90E2981B892F0895209190032223B2
:102D800021F021502093900325C020918F032F5FC5
:102D900020938F0325312CF010928E0310928F0315
:102DA0001BC020918C0330918D038217930739F05B
:102DB00020918E032F5F20938E0310928F0320911A
:102DC0008E0326304CF010928E0310928F0384E114
:102DD0008093900381E0089590938D0380938C03FA
:102DE00080E0089520918A0330918B038217930726
:102DF00059F0209189032F5F20938903253030F00B
:102E000090938B0380938A031092890380918A03A5
:102E100090918B030C94BD1686B123B1837030E181
:102E2000839FC00111242F70822B0895009789F091
:102E300025E0E6E9F3E0DC0101900D922A95E1F747
:102E400085E0E6E9F3E0A1E9B3E001900D928A950F
:102E5000E1F7089545E050E061E973E086E993E029
:102E60000E94341A0895EF92FF920F931F93CF930D
:102E7000DF93EC013B9A439A429A80E58A95F1F7F9
:102E80000E940C17182F43988091DD01823028F49E
:102E900018838FEF89838A832DC0429890E59A9595
:102EA000F1F70E940C17E82E429A80E58A95F1F717
:102EB000429890E59A95F1F70E940C17F82E429AE5
:102EC00080E58A95F1F7429890E59A95F1F70E948E
:102ED0000C17082F429A80E58A95F1F70E940C178B
:102EE000429890E59A95F1F7429A1883E9828A838D
:102EF000FB820C83DF91CF911F910F91FF90EF9098
:102F00000895CF93DF9300D000D01F92CDB7DEB7E6
:102F1000CE0101960E943317298120954A81409560
:102F20003B81309585E0E6E9F3E0DF011D928A956B
:102F3000E9F720FF06C081E090E09093980380932A
:102F4000970321FF09C080919703909198038260B5
:102F5000909398038093970322FF09C08091970371
:102F6000909198038460909398038093970323FF34
:102F700009C080919703909198038860909398037B
:102F8000809397036091DD01522F5071207262305F
:102F900008F45BC086E08093960344FF09C08091EB
:102FA000970390919803806490939803809397037C
:102FB000552349F0809197039091980380619093F5
:102FC000980380939703222349F08091970390916F
:102FD00098038062909398038093970345FF09C0FC
:102FE00080919703909198039460909398038093B5
:102FF0009703633009F042C032FF09C08091970304
:10300000909198038068909398038093970331FF81
:1030100009C08091970390919803916090939803D1
:103020008093970330FF09C0809197039091980394
:103030009260909398038093970333FF1FC0809111
:10304000970390919803986015C087E0809396034A
:10305000552349F080919703909198038061909354
:10306000980380939703222349F0809197039091CE
:1030700098038062909398038093970380E00F9069
:103080000F900F900F900F90DF91CF910895CF93F5
:10309000DF9300D000D01F92CDB7DEB73A9A429AA4
:1030A00084B1807F84B985B18F6085B987B18C7F09
:1030B00087B988B1836088B9CE0101960E94331721
:1030C00081E08093DD0189818F709A818F3089F44E
:1030D000892F8F70833069F48C818F70833021F455
:1030E0008D818F70833011F083E001C082E0809386
:1030F000DD0195FD03C083E08093DD010E9481170F
:1031000080E00F900F900F900F900F90DF91CF9174
:10311000089581ED91E00895CF93DF93CDB7DEB7A9
:10312000C054D1090FB6F894DEBF0FBECDBF80E604
:103130008BB98FEB8AB987EB9BE00197F1F700C061
:1031400000004E9903C081E08093E9018091E9017C
:10315000811108C087E088B983EC87B915B88FEF73
:1031600084B905C017B88FEF88B914B885B90E9423
:10317000620E0E94220C0E94740A5C010E941F0CC5
:10318000782E692E0E944E0E582E492E0E948918C4
:103190008C018091E901882329F0D801ED91FC91FF
:1031A0000995580140E0BE016C5E7F4F80E090E0E1
:1031B0000E94BA0F20E030E040E050E0BE01695DBF
:1031C0007F4FCE0144960E94AF0F8091E90181119B
:1031D0004AC00E94BD0C99278130910541F00297A9
:1031E00061F485E08093E8018CE291E03AC084E0EC
:1031F0008093E80182E391E034C08091E901882363
:1032000091F00E9489188C01DC011296ED91FC91DD
:1032100013970995D8011696ED91FC911797CE0159
:103220000196099520C00E94740A8C01DC01129657
:10323000ED91FC9113970995D8011696ED91FC91AB
:103240001797CE01019609958981823029F48093E0
:10325000E80186E291E005C083E08093E80180E226
:1032600091E00E94F10800E715E020E031E041E143
:10327000BE01695D7F4F88E391E00E9493080E9440
:10328000E1087894E12CF12C912CC12CD12C312C1B
:10329000812C00E010E098E0292E83B78E6083BF78
:1032A00083B7816083BF889583B78E7F83BF80910A
:1032B000EA018823E1F31092EA0189E89BE1019792
:1032C000F1F700C00000882021F091E08916C9F1D3
:1032D00054C0109277038091E901811120C0AFEFB3
:1032E000EA1AFA0AB9E7EB16F104CCF00E94BD0C19
:1032F0008130910561F0029719F0E12CF12C0FC09B
:10330000052D142DE12CF12C82E0382E06C0072D5E
:10331000162DE12CF12C3324339488248394A114AA
:10332000B10469F1D5011296ED91FC9113970995BD
:10333000D5011696ED91FC911797CE01019609954E
:103340001EC0D8011296ED91FC9113970995882320
:1033500041F0BFEFCB1ADB0A8BE0C816D104A4F012
:103360000CC0D8011696ED91FC911797CE010196ED
:103370000995992039F0939405C0812C05C09924B2
:10338000939402C0C12CD12C0E94EE0881112CC054
:103390008EEF0E947405823021F0833021F020E00E
:1033A00003C021E001C022E0492DBE016C5E7F4FC9
:1033B000CE01019621962FAF21970E94BA0F219638
:1033C0002FAD2197B2E0B9150CF4912C30E0432DCC
:1033D00050E0BE01695D7F4FCE0144960E94AF0F61
:1033E00061E1CE01879637C04091E801298130E044
:1033F000842F992787FD90952817390709F04DCF1D
:10340000433021F14CF4423009F047CF8C819D814B
:1034100099AF88AF62E01DC0443071F0453009F0CB
:103420003CCFFE013A96DE01D896822D01900D9296
:103430008A95E1F768E00DC08E819F81A885B985E6
:1034400088AF99AFAAAFBBAF64E003C08B8188AFF0
:1034500061E0CE01C8960E948C081FCFEE0FFF1FBF
:103460000590F491E02D0994FB01DC0104C08D91DD
:103470000190801921F441505040C8F7881B990BE6
:103480000895FB01DC0102C001900D9241505040B3
:10349000D8F70895DC0101C06D9341505040E0F72A
:1034A0000895DC01CB01FC01F999FECF06C0F2BD05
:1034B000E1BDF89A319600B40D9241505040B8F7F2
:1034C0000895DC01A40FB51F4150504048F0CB01D6
:1034D000840F951F2E910E94721A41505040D0F7D0
:1034E0000895262FF999FECF92BD81BDF89A0197D4
:1034F00000B4021639F01FBA20BD0FB6F894FA9A3C
:0A350000F99A0FBE0895F894FFCF6A
:10350A00E02080E02080E02080E0208000000000B1
:10351A00E02080E02080E02080E0208000000000A1
:10352A000000A42052080000A42052100000A42089
:10353A0052470000A42052640000A4200101650A39
:10354A00390A300A040A00000000000104070B0FC0
:10355A0013171B1F252B32393F45494D50535659D6
:10356A005C5E60616263640000000001020304069D
:10357A00080A0C0E10121920262C343C3D3E3F40FE
:10358A004142434445464748494A00010203060C62
:10359A0012161F2832383C404345464748494A00DC
:1035AA00000000000000000000001B0CF90AF00AED
:1035BA00A40AB80ACA0A054A0E1C0E000DF50C0028
:1035CA0000410E455854454E4D4F544500030000E6
:1035DA0000471881172A17161700000000024558DD
:0835EA0054454E4D4F544500BD
:00000001FF
